:020000040800F2
:1000000000070020210500082D160008AD15000886
:1000100005160008AD150008D915000823050008CD
:100020002305000823050008230500088137000880
:100030002305000823050008230500082305000800
:1000400023050008230500082305000823050008F0
:100050002305000823050008B53B0008E13B000824
:100060000D3C0008393C0008653C000823050008E9
:1000700023050008230500082305000823050008C0
:10008000230500082305000823050008A125000812
:100090000D26000861260008B5260008913C0008DE
:1000A0002305000823050008230500082305000890
:1000B000013A00082305000823050008230500086D
:1000C0002305000823050008230500082305000870
:1000D00023050008230500084D2900082305000812
:1000E000F93C000823050008230500082305000843
:1000F0002305000823050008230500082305000840
:10010000230500082305000823050008230500082F
:10011000230500082305000823050008230500081F
:10012000230500082305000823050008230500080F
:1001300023050008230500082305000823050008FF
:1001400023050008230500082305000823050008EF
:1001500023050008230500082305000823050008DF
:1001600023050008230500082305000823050008CF
:1001700023050008230500082305000823050008BF
:1001800023050008230500082305000823050008AF
:10019000230500082305000823050008230500089F
:1001A000230500082305000823050008230500088F
:1001B000230500082305000823050008230500087F
:1001C000230500082305000823050008230500086F
:1001D000230500082305000823050008230500085F
:1001E000D0400B1CD1409C46203AD3401843524289
:1001F00063469340184370479140031C90409C46CF
:10020000203A9340194352426346D3401943704702
:1002100053B94AB9002908BF00281CBF4FF0FF316D
:100220004FF0FF3000F07AB9ADF1080C6DE904CE63
:1002300000F006F8DDF804E0DDE9022304B07047C1
:100240002DE9F0478C460D460446089E002B51D1FF
:100250008A4217466DD9B2FA82FEBEF1000F0BD06A
:10026000CEF1200C01FA0EF520FA0CFC02FA0EF782
:100270004CEA050C00FA0EF44FEA174A250CBCFBB9
:10028000FAF81FFA87F90AFB18CC45EA0C4508FB77
:1002900009F3AB420AD9ED1908F1FF3280F023814E
:1002A000AB4240F22081A8F102083D44ED1AA4B20D
:1002B000B5FBFAF00AFB105544EA054400FB09F9C6
:1002C000A14509D9E41900F1FF3380F00A81A14565
:1002D00040F2078102383C44A4EB090440EA08409C
:1002E0000021002E61D024FA0EF4002334607360E4
:1002F000BDE8F0878B4207D9002E54D0002186E854
:1003000021000846BDE8F087B3FA83F1002940F0E8
:100310008E80AB4202D3824200F2FA80841A65EBEF
:1003200003050120AC46002E3FD086E81010BDE842
:10033000F08712B90127B7FBF2F7B7FA87FEBEF1D3
:10034000000F34D1EB1B3A0C1FFA87FC0121B3FBE1
:10035000F2F8250C02FB183345EA03450CFB08F3C1
:10036000AB4207D9ED1908F1FF3002D2AB4200F2DF
:10037000D1808046ED1AA3B2B5FBF2F002FB105516
:1003800043EA05440CFB00FCA44507D9E41900F13D
:10039000FF3302D2A44500F2B8801846A4EB0C0447
:1003A00040EA08409DE731463046BDE8F087CEF18F
:1003B000200405FA0EF307FA0EF720FA04F83A0CB7
:1003C00025FA04F448EA0308B4FBF2F14FEA1845B1
:1003D00002FB11441FFA87FC45EA044501FB0CF3BC
:1003E000AB4200FA0EF409D9ED1901F1FF3080F0AB
:1003F0008A80AB4240F2878002393D44EB1A1FFAF3
:1004000088F5B3FBF2F002FB103345EA034500FB2D
:100410000CF3AB4207D9ED1900F1FF386FD2AB42B4
:100420006DD902383D44EB1A40EA01418FE7C1F132
:10043000200722FA07F88B4005FA01F448EA030383
:1004400020FA07FE4FEA134CFD404EEA040EB5FBBE
:10045000FCF94FEA1E440CFB19551FFA83F844EAD5
:10046000054509FB08F4AC4202FA01F200FA01FA70
:1004700008D9ED1809F1FF3043D2AC4241D9A9F1B6
:1004800002091D442D1B1FFA8EFEB5FBFCF00CFB70
:1004900010554EEA054400FB08F8A04507D9E418BA
:1004A00000F1FF3529D2A04527D902381C4440EA83
:1004B0000940A4EB0804A0FB02894C45C6464D4602
:1004C00015D312D056B1BAEB0E0364EB050404FA4F
:1004D00007F7CB401F43CC40376074600021BDE874
:1004E000F0871846F8E69046E0E6C245EAD2B8EB57
:1004F000020E69EB03050138E4E72846D7E74046DA
:1005000091E78146BEE7014678E702383C4445E77B
:10051000084608E7A8F102083D442BE7704700BFF2
:1005200002E000F000F8FEE772B63A4880F308886F
:10053000394880F3098839484EF60851CEF2000157
:10054000086040F20000CCF200004EF63471CEF2AA
:1005500000010860BFF34F8FBFF36F8F40F20000C0
:10056000C0F2F0004EF68851CEF200010860BFF3F1
:100570004F8FBFF36F8F4FF00000E1EE100A4EF681
:100580003C71CEF200010860062080F31488BFF3AE
:100590006F8F03F071F903F051F903F097F94FF001
:1005A00055301F491B4A91423CBF41F8040BFAE702
:1005B0001C49194A91423CBF41F8040BFAE71A4919
:1005C0001A4A1B4B9A423EBF51F8040B42F8040BE7
:1005D000F8E700201749184A91423CBF41F8040B44
:1005E000FAE703F02FF903F0C5F9144C144DAC42AF
:1005F00003DA54F8041B8847F9E700F041F8114C7E
:10060000114DAC4203DA54F8041B8847F9E703F0B4
:1006100017B9000000070020002300200000000898
:100620000001002000070020604000080023002097
:10063000242300202823002090390020E001000816
:10064000E0010008E0010008E00100082DE9F04F9A
:100650002DED108AC1F80CD0C3689D46BDEC108A00
:10066000BDE8F08F002383F311882846A0470020BF
:1006700002F086FDFEE702F0EDFC00DFFEE7000081
:100680002DE9F04103F018F8804603F065F80546BF
:1006900000283DD12B4B98453AD0013398453AD0AC
:1006A000294B28F0FF029A4238D15FFA88F000F017
:1006B00051FA2E4642F2107400F060FC08B100249A
:1006C000264600F04DFA074660B36CBB374635B19D
:1006D0001E4B984503D003F037F80024274600202E
:1006E00002F0F4FF1A4B1B691B0420D40FB100F079
:1006F00031F800F09BFC00F08FFE00F099FF0546FA
:10070000BCB900F043FD4FF47A7002F03FFDF7E70B
:100710002E460024D0E704460126CDE706464FF4D6
:100720007A74C9E70446D2E74FF47A74CFE700241D
:10073000DFE700F07DFF401BA042E2D900F00AF89D
:10074000DBE700BF010007B0000008B0263A09B09F
:100750000004024010B51E4B1E4953F8042F01320D
:1007600000D110BD8B42F8D11B4C1C4B22689A4221
:100770002CD91B4B9B6803F1006303F580339A422D
:1007800024D202F0B5FF02F0C7FF002000F05EFEA9
:10079000144B0220187000F095FE134B1A6C0022C7
:1007A0001A64196E1A66196E596C5A64596E5A6633
:1007B0005B6E72B60D4A0E4B13601B6822682021D7
:1007C00081F311889D4683F30888104710BD00BF50
:1007D000FCFF00081C00010804000108FFFF0008DE
:1007E00000230020282300200038024008ED00E00C
:1007F0000000010809490B6849F269009AB21B0C14
:1008000000FB0233064A0B60136844F2506198B251
:100810001B0C01FB0030106080B2704720230020C9
:100820001C23002010B500211022044600F066FEB3
:10083000034B03CB206061601868A06010BD00BF4F
:10084000107AFF1FF0B51F4CBBB000F0F1FEA3689B
:10085000C31AF92B30D906AD2346A0602822002107
:10086000284601F0A3FB04F10E0000F03FFE002338
:10087000C6B2591D5F1CDBB2B3424FEAC10107DAB1
:100880000E3323440822284601F090FB3B46F0E754
:10089000012303930823207B02930B4B0193C1F3A5
:1008A000CF013023059100930146049503A3D3E9BA
:1008B0000023064801F0B4F93BB0F0BD78F6339F51
:1008C00093CACD8D68330020753300204433002057
:1008D00070B50D4614461E4601F04AF950B9022E75
:1008E0000ED1012C0CD112A3D3E90023C5E90023BA
:1008F000012070BD052C14D003D8012C09D0002094
:1009000070BD282C09D0302CF9D10BA3D3E90023DA
:10091000ECE70BA3D3E90023E8E70BA3D3E900231B
:10092000E4E70BA3D3E90023E0E700BFAFF30080C7
:10093000401DA12026812A0B78F6339F93CACD8DC6
:100940009E6AC421818A46EE26417272DF25D7B79E
:10095000F017304A39059E5638B504460D46034611
:1009600020222846002101F021FB22792346032A78
:1009700028BF032203F8042F28460222202101F079
:1009800015FB62792346072A28BF072203F8052FA3
:1009900028460322222101F009FBA2792346072AD7
:1009A00028BF072203F8062F28460322252101F03D
:1009B000FDFA284604F108031022282101F0F6FA76
:1009C000382038BD2DE9F04FFFB01FAE0CAD40F21E
:1009D000791280460F463046002100F08FFD4822F4
:1009E0000021284600F08AFD00F022FE574B4FF40C
:1009F0007A72B0FBF2F0186093E80700002485E8F3
:100A0000070001230DF152002B746C74FFF70AFFED
:100A1000512385F8213006AB18464D4985F8204012
:100A200003F00EFA152228643146284685F83C204A
:100A3000FFF792FF10AB044601460822304601F052
:100A4000B5FA0822A1180DF14103304601F0AEFAC3
:100A50000DF14203082204F11001304601F0A6FA1C
:100A600011AB202204F11801304601F09FFA12ABBD
:100A7000402204F13801304601F098FA14AB082204
:100A800004F17801304601F091FA0DF1510308228A
:100A900004F18001304601F089FA04F1880A0DF171
:100AA000520904F5847B4B465146082230460AF130
:100AB000080A01F07BFAD34509F10109F3D119AB1A
:100AC00008225946304601F071FA04F588744FF057
:100AD000000995F834304B4510D84FF0000995F8CF
:100AE0003C304B4515D92B6C21464B4408223046EF
:100AF00001F05CFA083409F10109F0E7AB6B21461B
:100B00004B440822304601F051FA083409F101093A
:100B1000DFE7E31DC3F3CF03F97E059300230496BB
:100B20000393BB7E0293193701230093019705A31A
:100B3000D3E90023404601F073F87FB0BDE8F08FA1
:100B4000AFF300809E6AC421818A46EE2C230020E8
:100B5000EC3E0008014B1870704700BF382300209E
:100B6000F0B5324B1C7B85B034B1314B0E221A816B
:100B70000024204605B0F0BD2E4A1068516802AB33
:100B800003C308230DEB03022B492C4803F03AF969
:100B9000054630B9264B2A480A221A8100F002FD88
:100BA000E6E70169B1F5E02F06D9214B25480B2274
:100BB0001A8100F0F7FCDCE7438B512B08D01C4A6C
:100BC00021480C2111815122194600F0EBFCD0E79D
:100BD0001E4A024402F11003994204D2144B1C48ED
:100BE00010221A81E5E710398E1A2046134900F0C9
:100BF00023FD3246074605F11801204600F01CFD92
:100C0000AB689F4202D1EB6898420AD0084B0D2294
:100C10001A8100903B46EA68A9680E4800F0C2FCC1
:100C2000A6E70D4800F0BEFC0124A2E768330020CF
:100C30002C230020503E0008DCFF060000000108C5
:100C4000583E0008643E0008763E00080800FFF7A2
:100C5000943E0008B13E0008DA3E00082DE9F04F4E
:100C6000ADB006AF80460C4600F082FF0646002875
:100C70005BD1237E022B19D1E38A012B16D100F020
:100C8000D7FC0546FFF7B6FD4FF4C873B54AB0FB75
:100C9000F3F105F5167501FB1300E37E15FA80F0FC
:100CA0001060914633B9B04B00221A709C37BD4694
:100CB000BDE8F08FA38AF5B2013BAB4206F1010615
:100CC0000CD93B1D691CC9001D4400950023082256
:100CD00001F0F801204601F03BF8EBE707F11400C2
:100CE000FFF7A0FD2A4607F11401381D03F07AF83A
:100CF00003460028D7D10F2D08D89B4B1D70D9F87B
:100D00000030A3F51673C9F80030CFE707F1980259
:100D1000014602F8950D20460092072201F018F8CE
:100D2000F978404600F01CFFC0E7E38A052B00F08D
:100D3000068106D8012BB9D121464046FFF742FE75
:100D4000B4E7282B3DD0302BB0D1637E874D0133E3
:100D50006A7BDBB29342E94640F0EF80E27E2B7B78
:100D60009A4240F0EA8007F19803002623F8846D48
:100D70001022009331460123204600F0E9FFB4F829
:100D80001480A8F102081FFA88F808F1030323F081
:100D900003030A3323F00703ADEB030D0DF1180A2B
:100DA00033469BB2B11C98454FEAC10106F10106DA
:100DB0006CDD5344009308220023204600F0C8FF56
:100DC000EEE7A38A013B9BB2C92B3FF66FAF674E9C
:100DD000357B4DBB06F10C03009308222B462946B8
:100DE000204600F0B5FFA38A05F10109013BEDB2F1
:100DF0009D424FEAC90109DA0E35354400950023BA
:100E00000822204600F0A4FF4D46ECE70023002214
:100E1000C6E900230023B36086F8D730C6F8D8307F
:100E2000337B0BB9E37E3373002507F114063B1DBA
:100E30000822294630467D60BD60FD6001F0B6F8AD
:100E40003B7A05F10109AB424FEAC90107D9FB68BA
:100E500008222B44304601F0A9F84D46F0E7C1F3D3
:100E6000CF010023E07E059104960393A37E0293B5
:100E70001934282301460093019438A3D3E90023B1
:100E8000404600F0CDFEFFF7DDFC0FE795F8D700F8
:100E900000F0E6FAD5F8D83006461BB995F8D70029
:100EA00000F0EEFAD5F8D83043449E4204D295F8CB
:100EB000D700013000F0E4FA4FEA980B0024A0B20A
:100EC000584504F1010408DA2B6880000AEB0001A0
:100ED0000122184400F01AFBF1E7D5E90023D5F808
:100EE000D84095F8D70012EB080243F100034444C0
:100EF000C5E90023C5F8D84000F0B2FA844209D30E
:100F000095F8D730013385F8D730D5F8D8309E1B07
:100F1000C5F8D860B8F1FF0F08DC00232B7300F090
:100F2000C1FAFFF71DFE08B1FFF714FC2B68104A49
:100F30009B0A013313810023AB60CD46B6E6BFF3B5
:100F40004F8F0C490C4BCA6802F4E0621343CB602C
:100F5000BFF34F8F00BFFDE7AFF3008026417272F1
:100F6000DF25D7B7403300203D3300206833002011
:100F70002C23002000ED00E00400FA0537B54FF007
:100F80000054214B22689A4229D1204B627D1A706D
:100F90001F48237D0373C9221E490E3000F09CFABE
:100FA000E0220021204600F0A9FA0125284603B0DE
:100FB00030BD0321184800F053FB8DE8030063683F
:100FC00083421ED1236899424FF0000319D1A360D8
:100FD0000E4B22691A70114BE2681A60E6E702F0C4
:100FE000C5FB054668B10E4A0E4C136C43F0007306
:100FF0001364A2680C4B9A4203D12369013B7E2BF8
:10100000D7D90025D2E700BF9AAD44C538230020C8
:101010006833002016000020586600401823002086
:1010200000380240506600405041A0B0F0B54B4A35
:101030004B4CD2F800E085B002236371BEF57A7F95
:101040004FF000030293ADF80C304AD3454B464DA8
:10105000B5FBFEF19E4594BF102309235A1CB1FB3A
:10106000F2F702FB171222B1022B3ADD013BDBB291
:10107000F4E77A1EB2F5806F33D2C3EBC306F21CDD
:10108000C2F3C702991A02F1010CC9B24FF47A7087
:1010900000FB0CF08C44B0FBFCF080B2B0F5617F3B
:1010A00006D9721E082692FBF6F2D2B29B1AD9B26A
:1010B000531E0F2B50D84B1E072B8CBF0023012330
:1010C000501800FB0770B5FBF0F5AE4509D143B1F0
:1010D0000123ADF808708DF80C308DF80A208DF8DA
:1010E0000B109DF80B30214921485A1E9DF80A30FB
:1010F000013B1B0443EA0253BDF80820013A1343A5
:101100004B6001F0E1FC002301931A4B00931A4954
:101110001A4B1B484FF4805200F0FAFC194B197817
:1011200011B1174800F01CFD00F082FA0546FFF7E8
:1011300061FB4FF4C87305F51675B0FBF3F202FBC3
:101140001300114B15FA80F0186002F005FB08B18E
:101150000F23238105B0F0BD0023B1E71823002041
:101160002C2300203F420F0040787D0110230020F7
:1011700080340020D10800083C2300205D0C0008CA
:101180004433002038230020403300202DE9F04F65
:1011900096A7D7E900670FF25C29D9E900898F4C3F
:1011A00093B0DFF858B2DFF858A2204600F082FD75
:1011B0000CAD079098B310220021284600F09EF94C
:1011C000079B197B4FF0000261F3030219468DF86B
:1011D000302051F8040F49680EAA03C21B680D9A0B
:1011E00063F31C029DF830300D9243F020038DF81C
:1011F000303000232A461946584601F075FC079006
:1012000030B9204600F05AFD079B8AF80030CCE741
:101210009AF80030072B40DC01338AF8003018229E
:101220000021284600F06AF9DFF8D0B1DFF8D4A138
:10123000002319462A46584601F07EFC014680BB31
:10124000102208A800F05AF9DAF8143083F4806309
:10125000CAF8143000F0EEF90B4612A9024611E963
:1012600003000DF1240E8EE803009DF83410C1F345
:10127000030089064CBF0E99BDF838108DF82C007C
:1012800046BFC1F31C0141F00041C1F30A010891BE
:10129000204608A900F0D2FECAE7204600F00EFD65
:1012A000BDE7204600F064FC824600284AD1DFF802
:1012B00058B100F0BDF9DBF80030984242D300F09D
:1012C000B7F90790FFF796FA079A8DF820A04FF428
:1012D000C87302F51672B0FBF3F101FB130012FAAA
:1012E00080F0CBF80000DFF824B19BF8001011B9B2
:1012F00001238DF8203028460791FFF793FA0799CC
:10130000C1F1100A5FFA8AFABAF1060F28BF4FF04E
:10131000060A524629440DF1210000F0DDF80AF1D9
:101320000103049308AB0393182302932C4B0193FE
:101330000123009332463B46204600F01BFC00236D
:101340008BF8003000F074F9264ADFF8C4A0136867
:10135000C31AB3F57A7F32D3106000F06BF90246FE
:101360000B46204600F0B4FC204600F001FC30B3F0
:101370009AF80C30DFF89CB0002B14BF0323022333
:101380008BF8053000F054F94FF47A732946B0FB1E
:10139000F3F0CBF800005846FFF7DEFA18230730C9
:1013A0000293114B0193C0F3CF0040F25513049008
:1013B0000093039542464B46204600F0DBFB9AF82B
:1013C0000C300BB1FFF73EFA9AF80C30002B7FF48B
:1013D000E8AE13B0BDE8F08FAFF3008044330020D7
:1013E0003C330020483400204C340020401DA12014
:1013F00026812A0BF1C6A7C1D068080F80340020CF
:101400004D34002000000240403300203D330020D6
:10141000683300202C23002070B502F01BF8094C23
:10142000094E2080002530682388834208D902F0C5
:101430000BF8336805440133B5F5803F3360F2D3D0
:1014400070BD00BF7C3400205034002002F0B2B8E0
:1014500000F10060920000F5803002F041B8000019
:10146000054B1A68054B1B889B1A834202D910440E
:1014700001F0EABF00207047503400207C34002087
:1014800038B5074D04462868204401F0E5FF28B927
:1014900028682044BDE8384001F0F6BF38BD00BFE1
:1014A00050340020064991F8243033B1002308223B
:1014B000086A81F82430FFF7CBBF0120704700BFD6
:1014C00054340020022802BF024B4FF480629A611C
:1014D000704700BF0000024010B50023934203D0C4
:1014E000CC5CC4540133F9E710BD0000024603464A
:1014F000981A13F9011B0029FAD1704702440346D8
:10150000934202D003F8011BFAE770472DE9F04738
:10151000234C94F8243005468846174683BB2E4654
:10152000DFF87C90C7B394F824302BB92022FF2138
:1015300048462662FFF7E2FF94F82400C0F1080550
:10154000BD4228BF3D465FFA85FAAD0041462A46B6
:1015500004EB8000FFF7C0FF94F82430A7EB0A07E4
:101560009A445FFA8AFABAF1080F2E44A844FFB2EF
:1015700084F824A0D6D1FFF795FF0028D2D108E047
:10158000266A06EB8306B042CAD0FFF78BFF00281D
:10159000C5D10020BDE8F0870120BDE8F08700BF7D
:1015A000543400200FB4002004B0704700B59BB045
:1015B000EFF3098168226846FFF78EFFEFF305839A
:1015C000044B9A6BDA6A9A6A9A6A9A6A9A6A9A6A6F
:1015D0009B6AFEE700ED00E000B59BB0EFF30981E8
:1015E00068226846FFF778FFEFF30583044B9A6B98
:1015F0009A6A9A6A9A6A9A6A9A6A9B6AFEE700BF2E
:1016000000ED00E000B59BB0EFF309816822684669
:10161000FFF762FFEFF30583034B5A6B9A6A9A6AEE
:101620009A6A9A6A9B6AFEE700ED00E0FEE7000016
:1016300001F0FEBF01F0E8BF30B5084D0A44914209
:101640000BD011F8013B09245840013CF7D040F37E
:1016500000032B4083EA5000F7E730BD2083B8ED4C
:101660002DE9F7431AA7D7E9006700EB81014FF096
:10167000FF324FF0FF330DF1040C884223D050F8B5
:1016800004EBCDF804E04FF0000E1EF80C800024AF
:101690004FEA086562406B404FF00908B8F1010855
:1016A0000BD0002A73F1000904DA92185B417240F2
:1016B0007B40F3E792185B41F0E70EF1010EBEF1BB
:1016C000040FE2D1D9E7D043D94303B0BDE8F0839A
:1016D0009336EAA9EBE1F0422DE9F047089E01F0CC
:1016E00007054FEAD60C2A4406F0070600EBD100A6
:1016F0004FF47F49954201D1BDE8F08705F0070E10
:1017000006F0070AD64577464FEAD50438BF574654
:10171000C7F10807511B0CEBD6088F42045D28BFA8
:101720000F4604FA0EF413F8081029FA07FE24FAFB
:101730000AF45FFA8EFE4C404EFA0AFE04EA0E04EA
:10174000614003F808103D443E44D3E70246006878
:1017500048B103681360D388118901339BB2994261
:10176000D38038BF1381704770B588B00D460446EA
:10177000202200216846FFF7C1FE20460495FFF7AE
:10178000E5FF054658B16B46044608AE1A4603CA43
:10179000B24220606160134604F10804F6D1284685
:1017A00008B070BD2DE9F041056885B90160BDE85C
:1017B000F081002B29DA930CB34229D1A54201D143
:1017C0000D60F3E7C8F800100C60BDE8F0814B68CD
:1017D00023F06047BE0C4FEAD37EC3F3807C16EA49
:1017E000230638BF3E46A8462C466368BEEBD37F2F
:1017F00023F06042DDD1974203D1C3F380739C454F
:101800000AD1974205E01C46EFE7B24206D01346E4
:101810009E422CBF00230123002BCFD12368A0467A
:10182000002BF0D12160BDE8F08100002DE9F041EE
:1018300006460F4600254FF6FF7441F221082A465E
:1018400030463946FEF7CCFCC0B284EA00240823B7
:1018500014F4004F4FEA4404A4B203F1FF3318BF5D
:1018600084EA080413F0FF03F2D10835402DE6D1D5
:101870002046BDE8F081000010B54B6833B9CA8A34
:1018800063F30902CA820020002110BDC4681A68EF
:101890001C60C360438A013B43824A60EDE700005D
:1018A00010B50A4441F22104914200D110BD11F853
:1018B000013B80EA0320082310F4004F4FEA400068
:1018C00080B203F1FF3318BF604013F0FF03F3D180
:1018D000EAE700002DE9F04F85B081468DE80A0067
:1018E000BDF83C409346002A00F0838024B10E9B53
:1018F000002B7ED0072C2AD809F10C00FFF726FF19
:10190000054628B96FF00205284605B0BDE8F08FFE
:1019100014220021FFF7F2FD22460E9905F108007E
:10192000FFF7DAFD631C2B749BF800302C4403F0A6
:101930001F0363F03F032372009B43F000436B607F
:10194000294609F11C00FFF72DFF0125DCE7019B6B
:101950001B0A4FF00008029300F10C034FF0800ABD
:101960004646454603930398FFF7F0FE07460028D6
:10197000C8D014220021FFF7C1FDC6BB9DF804307A
:101980003B729DF808307B7202220E9B711E194437
:10199000B4420AD9B8180132D2B211F801EF80F876
:1019A00008E00136072AB6B2F2D19BF8001001F028
:1019B0001F01B44208BF4FF0400AB81841EA48116D
:1019C0004AEA01030372009B013243F000437B604B
:1019D0003A74394609F11C00FFF7E4FE0135B442C0
:1019E0002DB288F001084FF0000ABCD18CE700222C
:1019F000CBE76FF0010587E72DE9F0471E46CB8A5C
:101A00009146C3F30902062A80460F4619D01346B1
:101A10000021B0B28DB25A1992B2052A09D9A84252
:101A200010D8FA8A034463F30902FA820120BDE860
:101A3000F087A842F3D93A4419F80140947601316D
:101A4000E8E70025FB8A7C68C3F30900821F1C239A
:101A5000B2FBF3FA03FB1A2A1FFA8AF27CB30121C4
:101A60002368002B39D1B31F03441C20B3FBF0F3D0
:101A700001339BB299420CD2BAF1000F09D1404612
:101A8000FFF764FE08B1C0F800A0206008B3044668
:101A90000022B6B24FF0000AB54230D2691E494466
:101AA0001346E01801339BB211F801EF80F804E00F
:101AB00001351C2BADB214D0AE42F2D8ECE7404653
:101AC000FFF744FE044608B1002303607C60002C4D
:101AD000DED16FF00200BDE8F087013189B21C460B
:101AE000BEE7AE42D8D94046FFF730FE08B1C0F895
:101AF00000A020600028ECD004460022CCE7FB8A3E
:101B0000C3F30902164466F30903FB828EE7000063
:101B1000F8B5044615460E46242200211F46FFF75D
:101B2000EDFC069B6360079B23626A094FF6FF7317
:101B30009A424FF0000028BF1A46A760207097B263
:101B400004F10C0503469A4205D100232B6027823D
:101B50006382A382F8BD2E60013335462036F2E75A
:101B600003781BB94BB2002BC8BF0170704700004F
:101B7000007870472DE9F7430D9EBDF828900B9D26
:101B80009DF83040BDF8388007461946104616B912
:101B9000B8F1000F40D11F2C3ED83B78D3B9B8F133
:101BA000070F36D839F0030336D1424631464FF697
:101BB000FF70FFF775FE4FEA092920F0010009F4D4
:101BC0004079400449EA0464400C44EA40244FF65A
:101BD000FF730DE043EA0923B8F1070F43EA0464F9
:101BE000F5D9FFF723FE42463146FFF759FE03467B
:101BF0008DE840012A4621463846FFF76BFE2B78D8
:101C00000133DBB21F2B88BF00232B7003B0BDE86C
:101C1000F0836FF00300F9E76FF00100F6E70000D2
:101C20002DE9F7430E9F0B9D9DF83480BDF83C6075
:101C300081469DF8300007B9AEBB1F2833D899F80C
:101C400000E0BEF1000F31D00C0244F080049DF89A
:101C5000281044EAC83444EA014444EA0E04072E3A
:101C600044EA00641CD919461046FFF7DFFD3246EE
:101C70003946FFF715FE0346019600972A4621468E
:101C80004846FFF727FEB8F1010F06D12B78013344
:101C9000DBB21F2B88BF00232B7003B0BDE8F0839D
:101CA0004FF6FF73E8E76FF00100F6E76FF003000F
:101CB000F3E70000C06900B104307047C3691A68D7
:101CC000C261C2681A60C360438A013B43827047A5
:101CD0002DE9F047D0F818A0DFF8708005461646C9
:101CE0001F4654464FF000090CB9BDE8F087D4E90F
:101CF0000223B21A67EB0303994508BF904523D22C
:101D0000AB699C42214628460FD1FFF7B5FDAB6970
:101D10001B68AB61EB6823606B8AEC60AC69013BCC
:101D20006B822346A2461C46DEE7FFF7A5FD23682B
:101D3000CAF80030EB6823606B8AEC60013B6B8271
:101D4000DAF800305446EDE72368EBE780841E00A4
:101D50002DE9F04F8BB00E4614460793DDF8508006
:101D60008346002800F01081B8F1000F00F00C81CC
:101D7000531E3F2B00F20881012A03D1079B002B41
:101D800040F00281BBF81450ED000023AE420893EE
:101D9000099304D3002630460BB0BDE8F08F331909
:101DA0009D42DBF80C303ABFAD1BEDB2254623B99E
:101DB000DBF81030002B00F093802F2E65D8C6F191
:101DC0003007BD424FF000032CBFFFB22F460093F7
:101DD000314608AB3A46DBF80800FFF77DFCA5EB7F
:101DE00007093E445FFA89F9BBF8143003F1005348
:101DF000063BDB000493DBF80C3003933021039B9C
:101E000013B1B9F1000F43D1DBF8100040B1B9F1C3
:101E1000000F05D0009708AB4A46711AFFF75CFC2B
:101E20002EB2002DB6D060070AD00AAB03EBD40166
:101E3000624211F8083C02F00702134101F8083C25
:101E4000082C54D9102C54D9202C8CBF08230423DF
:101E5000079A002A00F09E80B4EBC30F00F09D802B
:101E6000082C48D89DF82030621E23FA02F2D107D0
:101E700006D54FF0FF3202FA04F423438DF82030E8
:101E80009DF8203088F8003085E7A9460027ABE7A9
:101E9000049BE02B28BFE02306930B44B342059339
:101EA00015D9A3EB060AD145039800972CBF5FFA1A
:101EB0008AFACA46711A08AB52460430FFF70CFC86
:101EC0005744A9EB0A095644FFB25FFA89F9049B0B
:101ED000069A05999B1A0493039B1B6803938EE74C
:101EE00000932A4608AB3146DBF8080096E7012349
:101EF000AEE70223ACE7102C12D8BDF82030621EEA
:101F000023FA02F2D20706D54FF0FF3202FA04F4A8
:101F10002343ADF82030BDF82030A8F800303AE770
:101F2000202C0FD8089A631E22FA03F3DB0705D58D
:101F30004FF0FF3303FA04F414430894089BC8F8E5
:101F4000003028E7402C22D0DDE908AB621E504665
:101F50005946FEF745F9002100F0010050EA01035F
:101F60000DD0224601200021FEF746F9404261EBE8
:101F7000410140EA0A0041EA0B01CDE90801DDE92F
:101F80000823C8E9002306E76FF0010603E76FF0B6
:101F9000080600E7012C3FF473AF082C7FF670AF02
:101FA000102CB8D9202CEAD8C8E7000030B5402A58
:101FB00085B01FD8002A08BF01220024012A0294FC
:101FC000039419D11B788DF8083053070AD004AB5D
:101FD00003EBD205544215F8083C04F00704A34073
:101FE00005F8083C00910346002102A8FFF774FBA6
:101FF00005B030BD4022E0E7082AE3D9102A03D813
:102000001B88ADF80830E0E7202A02D81B6802934D
:10201000DBE7D3E90045CDE90245D6E710B5CB684B
:102020001BB98B600B618B8210BDC4681A681C6081
:10203000C360438A013B4382CA60F0E72DE9F04F59
:10204000D1F800908FB0C9F3C01604460D46CDE913
:102050000223002E50D0C9F3C03AC9F30626B9F1C5
:10206000000F80F2CB8119F0C04F40F0C7812B7B6D
:10207000002B00F0C381BAF1020F03D02278B242E4
:1020800040F0BF8109F07F02BAF1020F059236D10C
:1020900019F07F0FC9F30F2B01D10BF0030B2B4469
:1020A0007606059A93F8038046EA0A4646EA82468F
:1020B0005FEAD81346EA0B06049300F0A1800022E1
:1020C00000230EA961E90823059B00936768534626
:1020D0005A462046B847002800F08F80A7698FB97C
:1020E000314604F10C00FFF73FFB0746D0B96FF013
:1020F00002000FB0BDE8F08F4FF0020AAFE7C9F35E
:10210000074BCCE73B699E420DD03F68002FF9D1C9
:10211000314604F10C00FFF727FB07460028E6D004
:10212000A3693B60A761DDE90601FFF77FFBB88289
:10213000F97D08F01F06C1F38401711A89B20FFA04
:1021400081FED7E90223BEF1000FBCBF01F1200ED2
:102150000FFA8EFE52EA0301C9F3046900F05D81B3
:10216000DDE90201801A61EB030102460B46B64825
:102170000021994208BF9042C0F04F81049B002B80
:1021800048D0BEF1010F00F3488118F0400F41D054
:10219000DDE902230021C7E9022306A82022FFF778
:1021A000ADF9DDE90223CDE906232B1D08932B7B36
:1021B000ADF82EB0013BDBB2ADF82C309DF81430F9
:1021C0008DF833308DF830A0A3688DF831608DF82C
:1021D000329006A920469847FB7DC3F38402013262
:1021E00062F38603FB75FB8A6FF30903FB821B0A0C
:1021F0006FF3C713FB7500207BE76FF00B0078E7E8
:10220000A76917B96FF00C0073E73B699E428FD046
:102210003F68F6E7FB7DC8F34012B2EBD31F40F0F6
:10222000F380C3F38403B34240F0F18004992B7B25
:102230004FEA981200293BD012F001085CD1032B21
:1022400040F2E880DDE90223C7E902232B7BAE1DC3
:10225000033BDBB23246394604F10C00FFF7CCFBFE
:10226000002814DA39462046FFF706FBFB7DC3F34E
:102270008402013262F38603FB75FB8A68F309036B
:10228000FB821B0A68F3C713FB75032031E7AB8899
:102290003B832A7B033AD2B2B88A3146FFF700FB70
:1022A000FB7DB882DA43C2F3C01262F3C713A1E721
:1022B00012BB2E1D013BDBB23246394604F10C0045
:1022C000FFF79AFB002814DA39462046FFF7D4FAC4
:1022D000FB7DC3F38402013262F38603FB75049A2B
:1022E000FB8A62F30903FB82049A1B0A62F3C71399
:1022F000CAE72A7B013ACEE7F98AC1F30901013B1B
:102300000529DAB25AD8281D00239A420AD907EBC8
:10231000010E013110F801CB8EF81AC001330629E5
:10232000DBB2F2D1DDE902019342CDE9060107F10A
:102330001A01089138BF04337968099134BF5B19D9
:1023400000230A93FB8AADF82EB0C3F309031A44A5
:102350009DF814308DF833300023ADF82C208DF823
:1023600030A08DF831608DF832907B602A7BB88A7E
:10237000013A291DFFF794FA3B8BB882834203D1BF
:10238000A36806A920469847204606A9FFF746FEFF
:10239000FB7DB88AC3F38402013262F38603FB75C6
:1023A000FB8A6FF30903FB821B0A6FF3C713FB75EC
:1023B0003B8B984214BF112000209AE6D7F804E026
:1023C000BEF1000F18D00623DEF8000088B9C91A44
:1023D00005F1040800EB010CBCF11B0FC3B2A1D83E
:1023E00093429FD2F44418F8013B8CF8043001303A
:1023F000F0E71C338646E7E7734693E76FF0090082
:1024000077E66FF00A0074E66FF00D0071E66FF08A
:102410000E006EE66FF00F006BE6FB7D68F386033F
:102420006FF3C713FB7539462046FFF725FA049B67
:10243000002B7FF4AAAEFB7DC3F38402013262F36A
:102440008603FB75DEE600BF80841E002DE9F041A7
:10245000504EB04240F089804F4CDFF840E1256C8F
:1024600045F000752564256E45F000752566246EDF
:10247000846AD4F8007207EA0E0747F00107C4F82F
:102480000072D4F8005205EA0E0545F0010545EA50
:102490000121C4F80012002A69D00021C4F81C12DE
:1024A0000F46C4F80412C4F80C12C4F8141204EB5A
:1024B000C10501311C29C5F84072C5F84472F6D136
:1024C0004FF0000E4FF0010C964514D1826AD2F8FD
:1024D0000032B04223F00103C2F8003257D12E4B34
:1024E0001A6C22F000721A641A6E22F000721A66D8
:1024F0001B6EBDE8F0819F781D8817F0010F18BF93
:10250000D4F804820CFA05F11CBF41EA0808C4F8AB
:10251000048217F0020F1EBFD4F80C8241EA0808AB
:10252000C4F80C827F0742BFD4F814720F43C4F87A
:10253000147204EBC5055F68C5F840729F68C5F862
:102540004472D4F81C522943C4F81C120C330EF107
:10255000010EB9E7846A0021C4F81C12C4F8041201
:10256000C4F80C12C4F81412AAE7002AF2D1836A44
:102570000022C3F84022C3F84422C3F80422C3F85F
:1025800014220122C3F80C22C3F81C229EE7BDE8E6
:10259000F08100BF80340020003802400000FFFFBF
:1025A000184A916A08B58B688B6013F0010105D059
:1025B00013F00C0F14BF4FF480310121D80506D55C
:1025C00013F4406F14BF41F4003141F00201D8030D
:1025D00006D513F4402F14BF41F4802141F00401CB
:1025E000D3690BB107489847202383F31188002152
:1025F000054800F0F3FD002383F31188BDE808408F
:1026000001F0F2B8803400208834002038B5124C34
:10261000A36ADD68AA0712D05A6922F002025A6141
:10262000A36913B1012120469847202383F3118821
:1026300000210A4800F0D2FD002383F31188EB0645
:1026400006D5A36A1021D960236A0BB102489847C6
:10265000BDE8384001F0C8B8803400209034002034
:1026600038B5124CA36A1D69AA0712D05A6922F024
:1026700010025A61A36913B1022120469847202312
:1026800083F3118800210A4800F0A8FD002383F39A
:102690001188EB0606D5A36A10211961236A0BB1D4
:1026A00002489847BDE8384001F09EB880340020C9
:1026B0009034002038B50F4CA36A5D685D602A072E
:1026C0000AD5042222701A6822F002021A60636A94
:1026D00013B10021204698476B0706D5A36A996974
:1026E000236A13B1090403489847BDE8384001F054
:1026F0007BB800BF8034002010B50F4C204600F09E
:10270000D1F90E4BA3620B21132000F0B3F90B217A
:10271000142000F0AFF90B21152000F0ABF90B21CC
:10272000162000F0A7F9002320461A460E21BDE826
:102730001040FFF78BBE00BF8034002000640040D3
:10274000114B984210B5044609D1104B1A6C42F057
:1027500000721A641A6E42F000721A661B6EA36A47
:1027600001221A60A36A5A68D20707D562685168C5
:102770001268D9611A60064A5A6110BD0121082009
:1027800000F022FCEEE700BF803400200038024059
:102790005B87010003291AD8DFE801F0020A0F1451
:1027A000836A9B6813F0E05F14BF0120002070472C
:1027B000836A9868C0F380607047836A9868C0F342
:1027C000C0607047836A9868C0F30070704700204B
:1027D0007047000010B503291FD8DFE801F0021F81
:1027E0002327816A8B68C3F30163183301EB03135A
:1027F000107881061ED55468C0F30011490041EAE3
:10280000C40141F0040100F00F0058609068986026
:10281000D268DA6041F00101196010BD836A03F5E6
:10282000C073E5E7836A03F5C873E1E7836A03F5DC
:10283000D073DDE79488C0F30011490041EA4451A8
:10284000E1E7000001290CD003D3022910D00020B9
:102850007047836ADA68920701D1186903E00120A2
:102860007047836AD86810F0030018BF01207047D2
:10287000836AF2E710B539B9836AD96889071BD131
:102880001B699B0704D110BD012915D0022948D12D
:10289000816AD1F8C031D1F8C401D1F8C8411461BE
:1028A000D1F8CC41546120240C610C69A40717D1E4
:1028B0004C6944F0100412E0816AD1F8B031D1F8CB
:1028C000B401D1F8B8411461D1F8BC41546120245D
:1028D000CC60CC68A40703D14C6944F002044C617D
:1028E00011795C0864F304119C0864F345111171BB
:1028F00089064BBF91681189DB085B0D4CBF63F300
:102900001C0163F30A01137948BF916060F303036C
:1029100013714FEA10234FEA104058BF1181137012
:10292000508010BD024AD36843F0C003D3607047A3
:1029300000440040044B5A6810439A6858600AB13A
:10294000181D1047704700BFAC3400202DE9F0413E
:102950003D4ED6F85C52EF682B68DA059CB20CD578
:10296000202383F311884FF40070FFF7E3FF6FF427
:1029700080732B60002383F31188202383F3118855
:10298000DFF8C48014F02F0331D183F311883806A7
:1029900013D5210611D5202383F311882B4800F08D
:1029A00005FA002844DA0820FFF7C4FF4FF67F73CA
:1029B0003B40EB60002383F311887A060DD5630654
:1029C0000BD5202383F31188F26C336D9A4201D129
:1029D000336C7BBB002383F31188D6F86422D36861
:1029E0000BB110699847BDE8F04100F0FDBE230728
:1029F00012D014F0080F0CBF00208020E10748BF60
:102A000040F02000A20748BF40F04000630748BFE5
:102A100040F48070FFF78EFFA4066B6805D596F82A
:102A200060124046194000F063FA2C68A4B2A9E78E
:102A30006860BFE727F040073F0410203F0CFFF716
:102A400079FFEF60C6E700BFAC340020E43400201B
:102A500010B5054C054A0021204600F027FA044B2A
:102A6000C4F85C3210BD00BFAC340020252900083A
:102A70000044004000F1604300F01F02400903F5EC
:102A8000614309018000C9B200F1604083F800137E
:102A900000F5614001239340C0F880310360704726
:102AA000FFF72ABE00F108020123037082600023B1
:102AB000C26000F110024360026142618361C36140
:102AC000036243627047000010B52023044683F37D
:102AD0001188022303704160FFF732FE0423237044
:102AE000002383F3118810BD2DE9F0411F460446F1
:102AF0000D461646202383F3118800F10808237839
:102B0000052B0ED029462046FFF744FE48B120464B
:102B100032462946FFF75EFE002080F31188BDE8AB
:102B2000F0813946404600F03DFB0028E7D0002305
:102B300083F31188BDE8F0812DE9F0411F4604467A
:102B40000D461646202383F3118800F110082378E0
:102B5000052B0ED029462046FFF774FE48B12046CB
:102B600032462946FFF786FE002080F31188BDE833
:102B7000F0813946404600F015FB0028E7D00023DD
:102B800083F31188BDE8F081F8B5154682680669BF
:102B9000AA420B46816938BF8568761AB542044659
:102BA00007D218462A46FEF797FCA3692B44A36177
:102BB0000DE011D932461846FEF78EFCAF1B3A469F
:102BC000E1683044FEF788FCE2683A44A261A368F9
:102BD0005B1BA3602846F8BD18462A46FEF77CFC1E
:102BE000E368E4E783682DE9F04104469342154623
:102BF000266938BF85684069361AB5420F4606D245
:102C00002A46FEF769FC63692B4463610DE012D923
:102C10003246A5EB0608FEF75FFC4246B919E068AC
:102C2000FEF75AFCE26842446261A3685B1BA36042
:102C30002846BDE8F0812A46FEF74EFCE368E4E74B
:102C400010B50A440024C361029B006040608460A8
:102C5000C160816141610261036210BD08B5826992
:102C60004369934201D1826882B9826801328260ED
:102C70005A1C42611970426903699A4201D3C368C0
:102C80004361002100F09EFA002008BD4FF0FF30A4
:102C900008BD000070B5202304460E4683F311885A
:102CA000A568A5B1A368A269013BA360531CA361F9
:102CB00015782269934224BFE368A361E3690BB1ED
:102CC00020469847002383F31188284670BD31467B
:102CD000204600F067FA0028E2DA85F3118870BD1B
:102CE0002DE9F74F05460F4690469A46D0F81C90BE
:102CF000202686F311884FF0000B144664B122465B
:102D000039462846FFF740FF034668B95146284632
:102D100000F048FA0028F1D0002383F31188A8EBD3
:102D2000040003B0BDE8F08FB9F1000F03D00190AB
:102D30002846C847019B8BF31188E41A1F4486F389
:102D40001188DBE7C16081614161C3611144009B6F
:102D5000006040608260016103627047F8B504461C
:102D60000E461746202383F31188A568A5B1A368F2
:102D7000013BA36063695A1C62611E70236962692A
:102D80009A4224BFE3686361E3690BB12046984728
:102D9000002080F31188F8BD3946204600F002FA81
:102DA0000028E2DA85F31188F8BD000083694269E2
:102DB0009A4210B501D182687AB982680132826084
:102DC0005A1C82611C7803699A4201D3C3688361EB
:102DD000002100F0F7F9204610BD4FF0FF3010BD84
:102DE0002DE9F74F05460F4690469A46D0F81C90BD
:102DF000202686F311884FF0000B144664B122465A
:102E000039462846FFF7EEFE034668B95146284684
:102E100000F0C8F90028F1D0002383F31188A8EB53
:102E2000040003B0BDE8F08FB9F1000F03D00190AA
:102E30002846C847019B8BF31188E41A1F4486F388
:102E40001188DBE7026843681143016003B118474A
:102E5000704700001430FFF743BF00004FF0FF330E
:102E60001430FFF73DBF00003830FFF7B9BF000056
:102E70004FF0FF333830FFF7B3BF00001430FFF7D7
:102E800009BF00004FF0FF311430FFF703BF00000F
:102E90003830FFF763BF00004FF0FF323830FFF7E4
:102EA0005DBF000000207047FFF7D2BD37B50F4B64
:102EB0000360002343608360C360012304460374FE
:102EC000154600900B464FF4807200F15C011430FF
:102ED000FFF7B6FE00942B464FF4807204F5AE71F6
:102EE00004F13800FFF72EFF03B030BD043F0008A7
:102EF00038B5C36904460D461BB904210844FFF7E1
:102F0000A1FF294604F11400FFF7A8FE002806DA05
:102F1000201D4FF48061BDE83840FFF793BF38BDF6
:102F2000024B00221B605B609A60704714370020E0
:102F3000002303748268054B1B6899689142FBD299
:102F40005A68036042601060586070471437002070
:102F500008B5202383F31188037C032B05D0042BB1
:102F60000DD02BB983F3118808BD436900221A6084
:102F70004FF0FF334361FFF7DBFF0023F2E790E8F8
:102F80000C001A6002685360F2E70000002303742B
:102F90008268054B1B6899689142FBD85A680360A8
:102FA000426010605860704714370020054B196963
:102FB0000874186802681A6053601861012303746A
:102FC000FDF744BB1437002030B54B1C87B00546D5
:102FD0000A4C10D023690A4A01A800F01BF92846C0
:102FE000FFF7E4FF049B13B101A800F051F9236936
:102FF000586907B030BDFFF7D9FFF8E71437002054
:10300000512F000838B50C4D41612B6981689A68D1
:103010009142044603D8BDE83840FFF789BF1846FF
:10302000FFF7B4FF01232C61014623742046BDE85D
:103030003840FDF70BBB00BF14370020044B1A6863
:103040001B6990689B68984294BF002001207047DC
:103050001437002010B5084C236820691A682260D4
:103060005460012223611A74FFF790FF0146206922
:10307000BDE81040FDF7EABA1437002008B5FFF7A5
:10308000DDFF18B1BDE80840FFF7E4BF08BD000050
:10309000FEE7000010B50C4CFFF742FF00F0ACF863
:1030A00080220A49204600F031F8012344F8180C28
:1030B000037400F075FB002383F3118862B60448A3
:1030C000BDE8104000F044B83C3700202C3F000819
:1030D000343F000800F018B9EFF3118020B9EFF386
:1030E0000583202282F311887047000010B558B97B
:1030F000EFF30584C4F3080414B180F3118810BD04
:10310000FFF7BCFF84F3118810BD0000826002222B
:1031100002740022427470478368A3F17C0243F872
:103120000C2C026943F83C2C426943F8382C074ABE
:1031300043F81C2CC26843F8102C022203F8082C18
:10314000002203F8072CA3F1180070476506000859
:1031500010B5202383F31188FFF7DEFF002104461A
:10316000FFF750FF002383F31188204610BD0000B5
:10317000024B1B6958610F20FFF718BF143700205E
:10318000202383F31188FFF7F3BF000008B5014641
:10319000202383F311880820FFF716FF002383F311
:1031A000118808BD49B1064B42681B6918605A6016
:1031B000136043600420FFF707BF4FF0FF307047F4
:1031C000143700200368984206D01A6802605060E5
:1031D00059611846FFF7ACBE7047000038B5044689
:1031E0000D462068844200D138BD036823605C60CE
:1031F0004561FFF79DFEF4E7054B03F114025A61A8
:103200009A614FF0FF32DA6100221A62704700BF04
:1032100014370020F8B50361C2600E46054600F081
:1032200041FB1A4B19461F4651F8142F8A420DD103
:103230001862AE606A602A600A2E2CBF80190A30BC
:103240009D615D61BDE8F84000F01ABB1B6A9268A1
:10325000C41A341928BF3446A24202D9181900F002
:103260001DFB7B699A6894420CD8AC6098685A68D8
:103270002B60041B6A6015605D609C604FF0FF333B
:10328000FB61F8BDA41A1B68ECE700BF14370020EF
:1032900038B51C4B01685A6990421D460DD04468F0
:1032A0002160026800215460C16091688068014417
:1032B00091604FF0FF32DA6138BD1A4642F8141FB0
:1032C0004A605B6900219342C16003D1BDE8384088
:1032D00000F0DEBA9A6881680A449A602C6A00F0AD
:1032E000E1FA6A699268001B82420AD9111A092917
:1032F00098BF00F10A02286ABDE83840104400F087
:10330000CDBA38BD143700202DE9F041184D002703
:1033100005F114066C6900F0C5FA2A6AA368811ADF
:103320008B4216D813442B6294E80C001A60226872
:10333000D4F80C8053606B69E760B34201D100F0B0
:10334000A7FA87F311882069C047202383F31188E7
:10335000E0E76A69B24208D05B1A0A2B2CBFC0189A
:103360000A30BDE8F04100F099BABDE8F08100BF35
:103370001437002000207047FEE70000704700006F
:103380004FF0FF3070470000BFF34F8F024AD36801
:10339000DB03FCD4704700BF003C024008B5094B7A
:1033A0001B7873B9FFF7F0FF074B1A69002ABFBFFC
:1033B000064A5A6002F188325A601A6822F4806222
:1033C0001A6008BDD0380020003C02402301674548
:1033D00008B50B4B1B7893B9FFF7D6FF094B1A6959
:1033E00042F000421A611A6842F480521A601A6868
:1033F00022F480521A601A6842F480621A6008BD92
:10340000D0380020003C0240072870B513D80B4A82
:103410000B4C137863B90B4E4FF0006144F8231046
:1034200056F823500133082B2944F7D10123137098
:1034300054F8200070BD002070BD00BFF43800209B
:10344000D4380020543F0008014B53F82000704747
:10345000543F000808207047072810B5044601D9DA
:10346000002010BDFFF7D0FF064B53F8243018445E
:10347000C21A0BB9012010BD12680132F0D1043B11
:10348000F6E700BF543F0008072810B5044621D8CE
:10349000FFF77AFFFFF782FF0F4AF323D360C300E1
:1034A000DBB243F4007343F002031361136943F486
:1034B00080331361FFF768FFFFF7A6FF074B53F850
:1034C000241000F013F9FFF783FF2046BDE81040F9
:1034D000FFF7C2BF002010BD003C0240543F00086F
:1034E0002DE9F84312F00103154640D184182E4A05
:1034F00094423CD82D4B1B6813F0010337D02C4C61
:10350000FFF74CFFF323E360FFF73EFF40F2012794
:10351000032D01D9830713D0254C0F46401A40F2E2
:103520000118EB1B0B44012B00EB0706236924D881
:1035300023F001032361FFF74BFF0120BDE8F8836F
:10354000236923F44073236123693B43236151F8CA
:10355000046B0660BFF34F8FFFF716FF03689E42B0
:1035600008D0236923F001032361FFF731FF002016
:10357000BDE8F883043D0430CAE723F440732361B7
:10358000236943EA08032361B94637F8023B3380D5
:10359000BFF34F8FFFF7F8FE3688B9F80030B6B2A8
:1035A000B342BED0DDE700BF00000808003802408B
:1035B000003C0240084908B50B7828B153B9FFF721
:1035C000EDFE01230B7008BD23B1BDE80840087073
:1035D000FFF7FEBE08BD00BFD038002038B500F0B0
:1035E00061F9074B1A68824207D9064AD2E90045B9
:1035F000003445F10105C2E90045186038BD00BF3F
:10360000F83800200039002070B5FFF765FD064648
:10361000FFF7E4FF054BD3E90045241845F1000509
:103620003046FFF763FD2046294670BD0039002073
:1036300008B5FFF7E9FF4FF47A720023FCF7E8FDC5
:1036400008BD00BF10B50244064B0439D2B2904207
:1036500000D110BD441C00B253F8200041F8040F03
:10366000E0B2F4E750280040104B30B51C6F240442
:1036700007D41C6F44F400741C671C6F44F40044AE
:103680001C670B4C236843F4807323600244094B8E
:103690000439D2B2904200D130BD441C00B251F87E
:1036A000045F43F82050E0B2F4E700BF0038024066
:1036B000007000405028004007B5012201A90020F9
:1036C000FFF7C0FF019803B05DF804FB13B5044693
:1036D000FFF7F2FFA04206D002A9012241F8044DF3
:1036E0000020FFF7C1FF02B010BD000070470000CE
:1036F000074B45F255521A6002225A6040F6FF729B
:103700009A604CF6CC421A60024B01221A70704744
:10371000003000400C390020034B1B781BB1034BD9
:103720004AF6AA221A6070470C3900200030004087
:10373000034B1A6812B9034A12681A60704700BF37
:103740000839002074380240024B4FF080721A6032
:10375000704700BF7438024008B5FFF7E9FF024B1D
:103760001868C0F3407008BD0839002008B5FFF79D
:10377000DFFF024B1868C0F3007008BD0839002055
:10378000EFF3098305494A6822F001024A60683371
:1037900083F30988002383F31188704730EF00E03A
:1037A000202080F3118862B60B4B0C4AD96821F4B3
:1037B000E0610904090C0A430949DA60CA6842F069
:1037C0008072CA6007490A6842F001020A6010224A
:1037D000DA7783F82200704700ED00E00003FA0575
:1037E000F0ED00E0001000E010B5202383F3118815
:1037F0000E4B5B6813F4006314D0F1EE103AEFF354
:103800000984683C4FF08073E361094BDB682366F1
:1038100084F30988FFF712FC10B1064BA36110BDB9
:10382000054BFBE783F3118810BD00BF00ED00E0FE
:1038300030EF00E0770600087A06000870470000C5
:10384000FEE70000084A094B09498B4204D3094AA4
:103850000021934205D3704752F8040F43F8040B3C
:10386000F3E743F8041BF4E7804000089039002098
:1038700090390020903900207047000000F086B891
:103880004FF08043002258631A610222DA607047C9
:103890004FF080430022DA60704700004FF0804311
:1038A000586370474FF08043586A70474B684360D5
:1038B0008B688360CB68C3600B6943614B690362AB
:1038C0008B6943620B6803607047000008B51F4BAB
:1038D0001F481A6942F0FF021A611A6922F0FF02BA
:1038E0001A611A691A6B42F0FF021A631A6D42F0EC
:1038F000FF021A65174A1B6D1146FFF7D7FF1648DE
:1039000002F11C01FFF7D2FF144802F13801FFF762
:10391000CDFF134802F15401FFF7C8FF114802F12F
:103920007001FFF7C3FF104802F18C01FFF7BEFFE3
:103930000E4802F1A801FFF7B9FF0D4802F1C401DA
:10394000FFF7B4FFBDE8084000F0A4B8003802401B
:1039500000000240743F00080004024000080240DA
:10396000000C024000100240001402400018024007
:10397000001C024008B500F019FAFFF78BFBBDE808
:103980000840FFF7D5BE000070470000104B1A6CCE
:1039900042F001021A641A6E42F001021A660D4AE0
:1039A0001B6E936843F0010393604FF08043312214
:1039B0009A624FF0FF32DA6200229A615A63DA604B
:1039C0005A6001225A6108211A601C20FFF752B880
:1039D00000380240002004E04FF0804208B513692F
:1039E000D1680B40D9B2C9439B07116107D5202389
:1039F00083F31188FFF76EFB002383F3118808BD62
:103A000008B5FFF7E9FFBDE80840FFF7EDBE00008D
:103A10001E4B1A6962F0FF021A611A69D2B21A616A
:103A20004FF0FF301A695A69586100215A6959618B
:103A30005A691A6A62F080521A621A6A02F0805257
:103A40001A621A6A5A6A58625A6A59625A6A1A6C2F
:103A500042F080521A641A6E42F080521A661A6E50
:103A60000B4A106840F480701060186F00F44070CA
:103A7000B0F5007F1EBF4FF4803018671967536898
:103A800023F40073536000F071B900BF00380240A6
:103A9000007000403C4B3D4A1A643D4A4FF440419F
:103AA00011601A6842F001021A601A689207FCD588
:103AB0009A6822F003029A60334B19469A6812F012
:103AC0000C02FBD1186800F0F90018609A601A68BF
:103AD00042F480321A600B689803FCD54B6F43F0B8
:103AE00001034B67284B5A6F9207FCD5294A5A604D
:103AF0001A6842F080721A60254A53685804FCD54F
:103B0000214B1A4619688901FCD52349C3F8841052
:103B1000196841F08061196013681B01FCD51F4BC7
:103B200093600323C2F88C304FF00063C2F89430E6
:103B30001B4B1A681B4B9A421B4B21D11B4A116825
:103B40001B4A91421CD140F203121A60164A1368B4
:103B500003F00F03032BFAD10B4B9A6842F00202D9
:103B60009A609A6802F00C02082AFAD15A6C42F460
:103B700080425A645A6E42F480425A665B6E7047C5
:103B800040F20372E1E700BF003802400004001079
:103B90000070004004194002083000240094883866
:103BA000002004E011640020003C024000ED00E031
:103BB00041C20F41084A08B5536911680B4003F030
:103BC0000103536123B1054A13680BB1506898474C
:103BD000BDE80840FFF708BE003C01401039002056
:103BE000084A08B5536911680B4003F0020353619A
:103BF00023B1054A93680BB1D0689847BDE80840E7
:103C0000FFF7F2BD003C014010390020084A08B51A
:103C1000536911680B4003F00403536123B1054A53
:103C200013690BB150699847BDE80840FFF7DCBD48
:103C3000003C014010390020084A08B5536911685A
:103C40000B4003F00803536123B1054A93690BB19C
:103C5000D0699847BDE80840FFF7C6BD003C014069
:103C600010390020084A08B5536911680B4003F069
:103C70001003536123B1054A136A0BB1506A984788
:103C8000BDE80840FFF7B0BD003C014010390020FE
:103C9000174B10B55C691A68144004F478725A61C5
:103CA000A30604D5134A936A0BB1D06A98476006FD
:103CB00004D5104A136B0BB1506B9847210604D5FD
:103CC0000C4A936B0BB1D06B9847E20504D5094AB7
:103CD000136C0BB1506C9847A30504D5054A936C3F
:103CE0000BB1D06C9847BDE81040FFF77DBD00BF19
:103CF000003C0140103900201A4B10B55C691A686D
:103D0000144004F47C425A61620504D5164A136DCE
:103D10000BB1506D9847230504D5134A936D0BB131
:103D2000D06D9847E00404D50F4A136E0BB1506E66
:103D30009847A10404D50C4A936E0BB1D06E9847F6
:103D4000620404D5084A136F0BB1506F98472304DF
:103D500004D5054A936F0BB1D06F9847BDE810406A
:103D6000FFF742BD003C014010390020062108B594
:103D70000846FEF77FFE06210720FEF77BFE0621A0
:103D80000820FEF777FE06210920FEF773FE0621C4
:103D90000A20FEF76FFE06211720FEF76BFE0621B4
:103DA0002820BDE80840FEF765BE000008B5FFF713
:103DB0002FFE00F00BF8FEF773FEFFF775F8FFF724
:103DC000E3FDBDE80840FFF759BD000000230449AA
:103DD0001A465A50C8180833802B4260F9D17047F0
:103DE0001039002010B501390244904201D1002061
:103DF00010BD10F8013B11F8014FA342F5D0181B7C
:103E000010BD00002DE9F8430746884691461E463E
:103E10008BB10D46A8EB0500B54207EB000402D2BA
:103E20000020BDE8F883324649462046FFF7DAFF16
:103E300018B1013DEEE7BDE8F8832046BDE8F88300
:103E4000034611F8012B03F8012B002AF9D1704722
:103E500040A2E4F1646891064E6F20617070207397
:103E600069670A00426164206677206C656E67743A
:103E7000682025750A0042616420626F6172645F88
:103E800069642025752073686F756C6420626520F5
:103E900025750A0042616420667720646573637249
:103EA0006970746F72206C656E6774682025750A7E
:103EB00000426164206170702043524320307825B5
:103EC0003038783A307825303878203078253038D6
:103ED000783A3078253038780A00476F6F6420666A
:103EE00069726D776172650A000000006F72672E5B
:103EF0006172647570696C6F742E41524B5F4750EC
:103F00005300000000000000712E00085D2E000824
:103F1000992E0008852E0008912E00087D2E00089D
:103F2000692E0008552E0008A52E00086D61696EE7
:103F3000000000004C3F000858370020D038002017
:103F400001000000913000080000000069646C6509
:103F500000000000004000000040000000400000A1
:103F6000004000000000010000000200000002000C
:103F700000000200A000902A00000000AAAAAAAA3D
:103F800050000024FFFB00000077000000900900B3
:103F90000100000500000000AAAAAAA501000080F7
:103FA000FFEF000000000000000000000000000023
:103FB00000000000AAAAAAAA00000000FFFF00005B
:103FC00000000000000000000000000000000000F1
:103FD000AAAAAAAA00000000FFFF0000000000003B
:103FE000000000000000000000000000AAAAAAAA29
:103FF00000000000FFFF00000000000000000000C3
:104000000000000000000000AAAAAAAA0000000008
:10401000FFFF0000000000000000000000000000A2
:1040200000000000AAAAAAAA00000000FFFF0000EA
:104030000000000000000000000000000000000080
:104040000A00000000000000030000000000000063
:1040500000000000ECC1FF7F010000000000000034
:1040600051000000000000000000070000000000F8
:10407000640000000000000040420F00FE2A010022
:04408000D204000066
:00000001FF
